:1002320012010001DC0000107104880800010000B6
:10024200000109022E0001010060010904000004FE
:10025200DCA0B0000705810310000A0705010310A6
:10026200000A0705820240000A0705020240000A4E
:04002000120B6E222F
:10002400E524541FF54C7023AF0CEFC4540F540156
:10003400FFBF0105754A038003754A01E4F54B7B54
:10004400047A00794A7D02120BF122E54CB40111C5
:10005400E4F54AF54B7B047A00794A7D02120BF1F0
:1000640022E54C6402703EE5295403F549E5293044
:10007400E70DE54925E004FF12035B8F4D800AE597
:100084004925E0FF12035B8F4DE54D30E105754ACC
:10009400018003E4F54AE4F54B7B047A00794A7D58
:0800A40002120BF122120B6E97
:0100AC002231
:1000AD00E524541FF54A701FE52764014526701796
:1000BD00C2AFAF0CEF54EFF50CD2AF7B007A0079E5
:1000CD0000E4FD120BF122E54A64027034E5274588
:1000DD0026702EE5295403F549E52930E70DE5494C
:1000ED0025E004FFE4FD1203BA800AE54925E0FF8F
:1000FD00E4FD1203BA7B007A007900E4FD120BF1E6
:04010D0022120B6E41
:0101110022CB
:10011200E524541FF54A701FE52764014526701730
:10012200C2AFAF0CEF4410F50CD2AF7B007A00796E
:1001320000E4FD120BF122E54A64027034E5274522
:1001420026702EE5295403F549E52930E70DE549E6
:1001520025E004FF7D011203BA800AE54925E0FF8C
:100162007D011203BA7B007A007900E4FD120BF1E3
:0401720022120B6EDC
:010176002266
:10017700E527547FFF7D011202727B007A00790028
:06018700E4FD120BF12261
:10018D00E526F549E549B4010C7E027F327D127CEE
:10019D0000120BFF22E549B4020C7E027F447D2E36
:0901AD007C00120BFF22120B6E04
:0101B6002226
:1001B700AF0DEF5401F5497B047A0079497D0112AF
:0201C7000BF13A
:0101C9002213
:1001CA00E52745267016FBFAF9FD120BF1C2AFAF0F
:1001DA000DEF54FEF50DD2AF120BE522E5276401AF
:1001EA0045267019FBFAF9FD120BF1120BE5120BF9
:1001FA00EBC2AFAF0DEF4401F50DD2AF22120B6E79
:01020A0022D1
:0E020B00E4F5497B047A0079497D01120BF17C
:0102190022C2
:10021A00E5274526700EE52945287008FBFAF9FD01
:08022A00120BF122120B6E22EF
:100272008F498D4AAF0CEFC413540720E002C2AF7E
:100282007F037DD012057EE54A60034349807F02E9
:10029200AD4912057EAF0CEFC413540720E002D221
:0202A200AF2289
:1002A4008F4AAF0CEFC413540720E002C2AF7F03A0
:1002B4007DD812057EE54A60097F027D0112057E24
:1002C40080077F02E4FD12057EAF0CEFC4135407D0
:0602D40020E002D2AF227F
:1002DA008F498D4AAF0CEFC413540720E002C2AF16
:1002EA007F037DF312057E7F02AD4912057E7F02F0
:1002FA00AD4A12057EAF0CEFC413540720E002D2B8
:02030A00AF2220
:10030C008F49AF0CEFC413540720E002C2AF7F0338
:10031C007DFB12057E7F02AD4912057EAF0CEFC44A
:09032C0013540720E002D2AF22B5
:100335007F037DF412057E7F021205908F3B7F02BD
:10034500120590AD077C00ED7D00FCED253BFDE43D
:050355003CFCFEAF05B9
:01035A002280
:02035B00AD07EC
:10035D00AF0CEFC413540720E002C2AF7F031205A8
:10036D007E7F02120590AE0CEEC413540720E002FE
:02037D00D2AFFD
:01037F00225B
:10038000AE077F03EE2440FD12057E7F021205902A
:01039000224A
:02039100AE07B5
:10039300AF0CEFC413540720E002C2AF7F03EE2477
:1003A30080FD12057E7F02120590AE0CEEC413543D
:0603B3000720E002D2AFBA
:0103B9002221
:1003BA008D4EAE07AF0CEFC413540720E002C2AF54
:1003CA007F03EE2440FD12057E7F02AD4E12057EAC
:0D03DA00AF0CEFC413540720E002D2AF2295
:0803E7007F037DF612057E2262
:1003EF00AF0CEFC413540720E002C2AF7F037DF5BB
:1003FF0012057E7F021205907508008F097F021289
:10040F000590EFFEE42509F509EE3508F508AF0C68
:0E041F00EFC413540720E002D2AFAE08AF09BD
:01042D0022AC
:10042E00AF0CEFC413540720E002C2AF7F057DFD71
:10043E0012057E7F04120590750A008F0B7F041241
:10044E000590EFFEE4250BF50BEE350AF50AAF0C21
:0E045E00EFC413540720E002D2AFAE0AAF0B7A
:01046C00226D
:08046D008B3C8A3D893EAD077E
:10047500AF0CEFC413540720E002C2AF7F0312058F
:100485007E7F02120590EF20E00FAF0CEFC41354EE
:100495000720E002D2AF7F00227F037DF012057EA8
:1004A5007F021205908F417F021205908F41E54131
:1004B500D3953F4003853F41E4F540E540C3954171
:1004C50050197F02120590AB3CAA3DA93E8540829A
:1004D500758300EF121684054080E07F037DF212DC
:1004E500057EAF0CEFC413540720E002D2AFAF4135
:0104F50022E4
:0804F6008B4F8A508951AD07BC
:1004FE00AF0CEFC413540720E002C2AF7F03120506
:10050E007E7F021205907F037DF012057E7F02E44E
:10051E00FD12057E7F02AD5212057EE4F553E553C2
:10052E00C3955250197F02AB4FAA50A951855382E1
:10053E00758300121655FD12057E055380E07F036C
:10054E007DFA12057EAF0CEFC413540720E002D2E1
:03055E00AFAF52EA
:010561002277
:100562008F3B7F03AD3B12057E7F037DF112057E3B
:0C057200E53B70077F037DF212057E223E
:10065B00657070417772697465203D203078256232
:10066B00782E0A0043504C4420636F756E7465728C
:10067B002072656164206261636B203D20307825B8
:0C068B0062782C2030782562782E0A005E
:10057E00D2A1E42FFFE434FFFE8F82F583EDF0C2AB
:01058E00A1CB
:01058F002249
:10059000D2A1E42FFFE434FFFE8F82F583E0FFC297
:0105A000A1B9
:0105A1002237
:1005A2008F48D2A1AF0DEFC31330E00C7B057A0662
:1005B200795B85484D121853E5484480F580C29016
:1005C200D291D292C292D292E548547FF580C292E1
:0505D200D292C2A1223B
:1005D7008D48AB07AA06D2A1E4FFEBFD12057EEA20
:1005E700FD7F0112057EAF0DEFC31330E019E4FF65
:1005F700120590AD077F011205908F4E8D4D7B053B
:100607007A06796F121853E54830E006C2A4D290F3
:090617008004D2A4C290C2A12209
:100620008B458A468947900002121655FF333333B3
:1006300054F8FD1216A8E5F0C41354072DFF120557
:10064000A2AB45AA46A9479000031216D5FFAEF00B
:0B065000900005121655FD1205D72280
:1007D60052656164205265676973746572733A2065
:1007E6004F6666736574203D20307825782C204C42
:1007F600656E677468203D20307825782C20496E18
:10080600646578203D20307825782E0A0057726975
:100816007465205265676973746572733A204F6612
:1008260066736574203D20307825782C204C656EE3
:10083600677468203D20307825782C20496E6465E1
:1008460078203D20307825782E0A00446174613A7C
:0C085600200030782562782C20000A0079
:0E069700754A217B047A00794A7D01120BF12D
:0106A5002232
:1006A600AE2AAF2B74802527F974003526A801FCE5
:1006B6007D017B047A0079331216237883E6FC08E1
:1006C600E6FDECFBAF05EF18F6EB08F67880E6FCE6
:1006D60008E6FDECFBAF05EF18F6EB08F6D37884D9
:1006E600E6940018E694404004120B6E22AF0DEF1C
:1006F600C4540F5403700CC2AFAF0DEF4408F50D90
:10070600D2AF22C2AFAF0DEF54CF4420F50DD2AF1A
:0107160022C0
:10071700E52430E743AF0DEFC31330E01B7B057AC9
:100727000779D685264D85274E852A4F852B5085F7
:100737002851852952121853E529B47217E528B4B0
:100747000412E5274526700CE52B6401452A700441
:1007570012069722120B6E22AF0DEFC31330E04F34
:100767007B057A08791385264D85274E852A4F857F
:100777002B508528518529521218537B057A087901
:1007870051121853E4F549C3E549952BE4952A50CE
:10079700157B057A08795874332549F8E6F54D1223
:1007A7001853054980E17B057A087960121853E5EB
:1007B70029B47117E528B40412E5274526700CE51E
:0E07C7002B6406452A70041206A622120B6E41
:0107D5002201
:100D4800486F73745F746F5F6465766963650044A8
:100D580065766963655F746F5F686F737400446577
:100D68007669636500496E746572666163650045FE
:100D78006E64706F696E74283029004F74686572EC
:100D8800005374616E6461726400436C6173730034
:100D980056656E646F72005265736572766564009D
:100DA8004745545F53544154555300434C454152B1
:100DB8005F464541545552450052455345525645A4
:100DC80044005345545F46454154555245005245E9
:100DD800534552564544005345545F414444524597
:100DE8005353004745545F44455343524950544F69
:100DF80052005345545F44455343524950544F524F
:100E0800004745545F434F4E464947555241544960
:100E18004F4E005345545F434F4E46494755524144
:100E280054494F4E004745545F494E544552464138
:100E38004345005345545F494E5445524641434546
:100E48000053594E435F4652414D450052657175F6
:100E58006573742054797065203D2025732C2052C9
:100E6800657175657374203D2025732E0A005265DF
:100E780071756573742054797065203D2025732C35
:100E8800206252657175657374203D203078256243
:100E9800782E0A000A50444955534244313220659D
:100EA80076616C756174696F6E20626F617264201F
:100EB8006669726D776172652056322E302E0A008F
:100EC800436F7079726967687420286329205068B5
:100ED800696C6970732053656D69636F6E647563BF
:100EE800746F72732C20313939382E0A0052652DEF
:100EF800636F6E6E656374205044495553424431A4
:100F080032206576616C756174696F6E20626F61FD
:100F1800726420746F205553422E0A00436F6E741A
:100F2800726F6C207374617465203D205553425F65
:100F380049444C452E00436F6E74726F6C20737475
:100F4800617465203D205553425F524543454956DB
:100F5800452E00436F6E74726F6C207374617465F4
:100F6800203D205553425F5452414E534D49542E13
:100F78000020436F6E74726F6C446174612E774306
:100F88006F756E74203D2025782E0A00456E6470BA
:100F98006F696E742034202842756C6B204F75740D
:100FA8002920537461747573203D202562782C20A4
:100FB800456E64706F696E742035202842756C6BBD
:100FC80020496E2920537461747573203D20256271
:100FD800782E0A00444D415F5374617465203D20AA
:100FE800444D415F49444C452E0A00444D415F53EE
:100FF80074617465203D20444D415F52554E4E4901
:101008004E472E0A00444D415F5374617465203D7C
:1010180020444D415F50454E44494E472E0A0043F7
:10102800504C4420636F756E7465722072656164FC
:10103800206261636B203D2030782562782C203057
:10104800782562782E0A004C6173742044657669AD
:10105800636520526571756573743A20626D5265D7
:10106800717565737454797065203D2030782562F8
:10107800782C2062526571756573743D203078252F
:1010880062782C207756616C7565203D2030782574
:10109800782C20774C656E677468203D2030782561
:1010A800782C2077496E646578203D203078257843
:1010B8002E0A00446174613A200030782562782C49
:1010C80020000A00566572626F7365204D6F646573
:1010D800203D204F4E2E0A00566572626F736520C0
:1010E8004D6F6465203D204F46462E0A00427573B9
:1010F800207265736574210A0053757370656E6498
:10110800206368616E6765210A005761697420660B
:101118006F722031207365636F6E64202E2E2E0A45
:10112800000500240500AD0500200501120500207A
:1011380005017705018D0500200501B70501CA05E0
:10114800020B05021A0500200500200500200500F5
:1011580020050020050020050020050020050020AE
:1011680005002005002005002005002005002005B9
:1011780000200500200507170500200500200500B0
:1011880020050D48050D57050D66050D6D050D77F4
:10119800050D83050D89050D92050D98050D9F0513
:1011A8000DA8050DB3050DC1050DCA050DD6050D14
:1011B800DF050DEB050DFA050E09050E1B050E2DB5
:0611C800050E3B050E4977
:0311CE0001230FEB
:100862008F478D48E547C4135407F5477048E5475D
:1008720075F003A4249BF582E43411F583E493FB21
:10088200740193FA7402938B4D8A4EF54FE54875C5
:10089200F003A424A7F582E43411F583E493FB74F6
:1008A2000193FA7402938B508A51F5527B057A0EAA
:1008B200795412185322AF0DEFC31330E02BE547E2
:1008C20075F003A4249BF582E43411F583E493FBD1
:1008D200740193FA7402938B4D8A4EF54F854850FA
:0A08E2007B057A0E79761218532276
:1008EC005389F0438901E4F58AF58CD2A9D28CD2D4
:0408FC00B9D2AF229C
:07090000C288D2A8C2B82290
:0A0907007580FF7590FF75A0FF22B8
:10091100759852438780758920758869758DF32292
:0109210022B3
:100922007543011209071209111208EC1209007B22
:10093200057A0E799C1218537B057A0E79C8121823
:10094200537B057A0E79F5121853120B9BE543700F
:1009520003020B69AF0CEF30E014C2AFAF0CEF54DF
:10096200FEF50CD2AFAF0DEF30E003120C762098FB
:1009720003020AF4121B43EF24F37003020ABD249C
:10098200A4601424F37003020AC224046003020A5E
:10099200F41203E7020AF4AF0CEFC4131354035426
:1009A20003700B7B057A0F79241218538030AF0C39
:1009B200EFC4131354035403FFBF020B7B057A0FDA
:1009C200793E1218538017AF0CEFC413135403541B
:1009D20003FFBF01097B057A0F795B1218537B0570
:1009E2007A0F7979852E4D852F4E1218537F041276
:1009F2000391C0077F051203918F4ED04D7B057A7C
:100A02000F7994121853AF0DEFC4540F5403700BA7
:100A12007B057A0F79DC121853802CAF0DEFC4548A
:100A22000F5403FFBF010B7B057A0F79F3121853A2
:100A32008015AF0DEFC4540F5403FFBF02097B05AD
:100A42007A10790D121853D2A1E4FF120590C00753
:100A52007F011205908F4ED04D7B057A10792712B7
:100A62001853C2A17B057A10794F85244D85254EF6
:100A720085264F852750852A51852B5285285385F7
:100A820029541218537B057A1079BB121853E4F5D6
:100A920044C3E544952BE4952A50157B057A1079D9
:100AA200C274332544F8E6F54D121853054480E12B
:100AB2007B057A1079CA1218538037120B9B803249
:100AC200AF0DEFC31320E0167B057A1079CC121814
:100AD20053C2AFAF0DEF4402F50DD2AF80147B05C8
:100AE2007A1079E0121853C2AFAF0DEF54FDF50D35
:100AF200D2AFAF0CEFC31330E014C2AFAF0CEF5460
:100B0200FDF50CD2AF7B057A1079F5121853AF0CB4
:100B1200EF1313543F30E017C2AFAF0CEF54FBF5A5
:100B22000CD2AF120B6D7B057A117901121853AFFB
:100B32000CEF131313541F30E00EC2AFAF0CEF547F
:100B4200F7F50CD2AF120CEFAF0DEF131313541FC6
:100B520020E00302094FC2AFAF0DEF54F7F50DD2FB
:0A0B6200AF120CBC02094F1209216A
:010B6C002266
:010B6D002265
:0F0B6E00E4FF7D011203BA7F017D011203BA2259
:080B7D007F067D431202DA221B
:100B8500C2AFE4F50CF50DD2AF7F4012030C7F1612
:060B95007D431202DA228A
:100B9B00C2B4C2B5120B7D7B057A117912121853B0
:100BAB00851148851047850F46850E457F147E00BD
:100BBB007D007C00121747AF48AE47AD46AC4512DF
:100BCB00170F121747AF11AE10AD0FAC0E12172245
:090BDB0040DA120B85D2B4D2B548
:010BE40022EE
:050BE500E4FF1202A470
:010BEA0022E8
:060BEB007F011202A422AA
:0E0BF100EDD3941050077F018D521204F622AE
:100BFF008E4A8F4BE4F52EF52FD3E52D9DE52C9CDA
:100C0F0040048C2C8D2D753005854A31854B32C3B0
:100C1F00E52D9410E52C940040277F01AB30AA31CD
:100C2F00A9327552101204F67410252FF52FE435E2
:100C3F002EF52EC2AFAF0CEF543F4440F50CD2AFA0
:100C4F00227F01AA4AA94B7B05852D521204F6E596
:100C5F002D252FF52FE52C352EF52EC2AFAF0CEF2E
:070C6F00543FF50CD2AF2247
:100C7600A2A682A5E433F52253220FE5226523605E
:100C86000E7F037B047A0079227552011204F685E1
:100C96002223AF0DEF1313543F30E019C2AFAF0D4F
:100CA600EF54FBF50DD2AF7889E6FF13B392B4EF9C
:050CB600A2E1B392B5BC
:010CBB002216
:100CBC007B017A007980120620C2AFAF0DEF54CFC2
:100CCC004410F50DD2AF7B007A007900E4FD120BD5
:100CDC00F17885E630E0067F0F12030C227F0712B5
:030CEC00030C22D4
:100CEF00E5245460F545E525540FF546AF45FD1253
:100CFF000862E545701DE54675F003A42429F582C9
:100D0F00E43411F583E493740193FA740293F912A6
:100D1F00178622E545B4401DE54675F003A4245916
:100D2F00F582E43411F583E493740193FA7402931A
:080D3F00F912178622120B6E57
:010D47002289
:0611D100040E0000000006
:03000B000211D807
:1011D800C0E0C0F0C083C082C0D0C000C004C00559
:1011E800C006C007C2AFAF11AE10AD0FAC0E1217DC
:1011F800477F017E007D007C0012170F8F118E1033
:101208008D0F8C0EAF0CEF4401F50CD2AFD007D088
:1012180006D005D004D000D0D0D082D083D0F0D072
:02122800E032B2
:0300030002122ABC
:10122A00C0E0C0F0C083C082C0D0C000C001C0020C
:10123A00C003C004C005C006C007C2AF121266D2FE
:10124A00AFD007D006D005D004D003D002D001D049
:0C125A0000D0D0D082D083D0F0D0E032A1
:10126600AF0CEF4420F50C1203358E398F3AE53A70
:1012760045396055E53A30E60C1212D7AF0CEF440B
:1012860002F50C8044E53930E003121485E53A3066
:10129600E707AF0CEF4404F50CE53A30E10312130F
:1012A600E9E53A30E0031212D8E53A30E3031214C6
:1012B600A1E53A30E2031214A7E53A30E503121429
:1012C600C5E53A30E4031214CBAF0CEF54DFF50C4E
:0112D60022F5
:0112D70022F4
:1012D800E4FF120380EF20E50302139CE4F52CF5EC
:1012E8002DF52EF52FFF7B047A007924753F08121F
:1012F800046DEF64086016E4FF7D011203BA7F01F4
:101308007D011203BAAF0CEF543FF50C22E526FD20
:10131800E527F526EDF527E528FDE529F528EDF57E
:1013280029E52AFDE52BF52AEDF52BE4FF120562E8
:101338007F01120562852A2C852B2DE4F52EF52FC9
:10134800E52430E70FAF0CEF4408F50CAF0CEF5471
:101358003FF50C22E52B452A700FAF0CEF4408F53A
:101368000CAF0CEF543FF50C22D3E52B9406E52A7D
:1013780094004016AF0CEF543FF50CE4FF7D0112CA
:1013880003BA7F017D011203BA22AF0CEF543F4428
:1013980080F50C22AF0CEFC41313540354036402FA
:1013A8007037FF7433252FF9E4FA7B04753F101268
:1013B800046DEF252FF52FE4352EF52EBF100BC346
:1013C800E52F952DE52E952C4016AF0CEF4408F52A
:1013D8000CAF0CEF543FF50C22AF0CEF543FF50C5B
:0113E80022E2
:1013E900C3E52D952FF53CE52C952EF53B7F011294
:1013F9000380AF0CEFC41313540354036401707BCF
:10140900C3E53C9410E53B6480948040297F01AB9F
:1014190030E532252FF9E531352EFA7552101204CF
:10142900F67410252FF52FE4352EF52EAF0CEF5459
:101439003F4440F50C22E53C453B60287F01AB3039
:10144900E532252FF9E531352EFA853C521204F69D
:10145900E53C252FF52FE53B352EF52EAF0CEF5446
:101469003FF50C22E53C453B70117F01FBFAF9F58C
:0B147900521204F6AF0CEF543FF50CCC
:011484002245
:10148500AF0DEFC4540F5403FFBF0208AF0DEF4477
:0C14950008F50D22AF0DEF54CFF50D222D
:0614A1007F03120380220C
:1014A7007F021203807F027B017A007986753F10E5
:0D14B70012046DEF6007AF0DEF4404F50D5A
:0114C4002205
:0614C5007F0512038022E6
:0614CB007F0412038022E1
:030000000214D116
:0C14D100787FE4F6D8FD758195021518AF
:10155D00E709F608DFFA8046E709F208DFFA803E70
:10156D0088828C83E709F0A3DFFA8076E309F60819
:10157D00DFFA806EE309F208DFFA806688828C83D9
:10158D00E309F0A3DFFA805A89828A83E0A3F60883
:10159D00DFFA804E89828A83E0A3F208DFFA804267
:1015AD0080AE80B480BA80C480CA80D080DA80E4F6
:1015BD0080378023805389828A83ECFAE493A3C811
:1015CD00C582C8CCC583CCF0A3C8C582C8CCC583A1
:1015DD00CCDFE9DEE7800D89828A83E493A3F608E8
:1015ED00DFF9ECFAA9F0EDFB2289828A83ECFAE0AF
:1015FD00A3C8C582C8CCC583CCF0A3C8C582C8CC4E
:10160D00C583CCDFEADEE880DB89828A83E493A39D
:10161D00F208DFF980CC88F0ED14B4040050C32437
:10162D001E83F582EB14B4050050B7241583258273
:10163D00F582EF4E60ACEF60010EE5829015AD7353
:08164D00000402000C0600126B
:10165500BB020CE58229F582E5833AF583E0224059
:1016650003BB0406E92582F8E622400DE58229F54B
:0F16750082E5833AF583E49322E92582F8E222A5
:10168400F8BB020DE58229F582E5833AF583E8F09B
:10169400224003BB0406E92582C8F6225005E92549
:0416A40082C8F222E4
:1016A800BB020A89828A83E0F5F0A3E0224003BBEB
:1016B800040687F009E71922400C89828A83E4939B
:0D16C800F5F074019322E3F5F009E3192217
:1016D500BB0210E58229F582E5833AF583E0F5F052
:1016E500A3E0224003BB0409E92582F886F008E659
:1016F50022400DE5832AF583E993F5F0A3E99322CA
:0A170500E92582F8E2F5F008E2227F
:10170F00EF2515FFEE3514FEED3513FDEC3512FC0C
:03171F0002176E40
:10172200C3EF9515F8EE951448F8ED951348F8ECCB
:10173200951248F892D5D082D083121766E8A2D5C6
:05174200C083C08222FB
:10174700E51605166010D0F0D0E0C012C013C01423
:10175700C015C0E0C0F08F158E148D138C1222AF08
:1017670015AE14AD13AC12E516146010D0F0D0E02E
:0F177700D015D014D013D012C0E0C0F015162238
:061786008A838982E473EE
:1017F100E559244DF8E6055922784A300702784D1B
:10180100E475F0011217BB02178C2000EB7F2ED27A
:10181100008018EF540F2490D43440D4FF30040BCF
:10182100EF24BFB41A0050032461FFE55A6002158A
:101831005A055DE55D7002055C30070D784AE47577
:10184100F0011217BBEF0217A7021B4D7403D20759
:101851008003E4C207F5598B4A8A4B894CE4F55A57
:10186100F55CF55DE55A60077F2012182C80F5F5CF
:101871005BC201C200C202C203C205C206C2081293
:1018810017FAFF700D3007057F0012183DAF5DAEEE
:101891005C22B42561C2D5C2041217FAFF24D0B468
:1018A1000A00501C75F00A20D50DC55AA4255AF519
:1018B1005A7002D20380E0C55BA4255BF55B80D73B
:1018C10024CFB41A00EF5004C2E5D204021A36D272
:1018D1000180C2D20080BED20280BAD2D580B8D2F5
:1018E1000580B27F2012182C2002077401B55A001E
:1018F10040F11217F1FF12182C021865D208D20616
:1019010080931217F1FB1217F1FA1217F1F94A4BF2
:10191100700679027A1B7B05200233E55A602FAFEE
:101921005BBF00011F7E008E827583001216556019
:10193100050EEE6F70F1C2D5EBC0E0EAC0E0E9C080
:10194100E0EE121A7AD0E0F9D0E0FAD0E0FB1217FB
:101951008CFF60A5EBC0E0EAC0E0E9C0E012182C02
:10196100D0E02401F9D0E03400FAD0E0FBE55B607F
:10197100DDD55BDA80837B057A1A7976D20280988D
:10198100791080027908C206C2088008D2D5790A86
:101991008004790AC2D5E4FAFDFEFF1217F1FC7B3F
:1019A100082001131217F1FD7B1030000A1217F104
:1019B100FE1217F1FF7B20EC3382D592D55013C371
:1019C100E43000069FFFE49EFEE42001039DFDE458
:1019D1009CFCE4CBF8C201EC700CCFCECDCCE8245A
:1019E100F8F870F38017C3EF33FFEE33FEED33FDEC
:1019F100EC33FCEB33FB994002FB0FD8E9EB3001F0
:101A010005F8D0E0C448B201C0E00AEC4D4E4F7871
:101A1100207B0070C2EAC0E0121A7CD0F0D0E02036
:101A21000104C4C0E0C4B201C0F0121815D0F0D551
:101A3100F0EB0218651217CB19035319815818D40A
:101A41004C18D04219854F198D44198D4918E94315
:101A51001993551977461977451977471B26501859
:101A6100D82D18DC2E18FF2B18E02318FD201B1190
:101A71002A000018F73F3F3F00790AA2D52003143E
:101A8100300509B910020404B9080104A2D52006E1
:091A9100025001042002669202D9
:101A9A00B55A005032C0E07F203003177F30A202CF
:101AAA0072067205500D121AD1C202C206C2057F11
:101ABA0030800F300503E9C0E012182C300503D03E
:101ACA00E0F9D0E0B55ACE3005177F30B9100C12C4
:101ADA00182C7F583004077F788003B9080312183E
:101AEA002C3002057F2D02182C7F202008F87F2B2E
:101AFA002006F322920280CF286E756C6C29002D85
:101B0A004958504443D2011217F13001F8C2017802
:101B1A005A30D504D200785BF60218961217F1B43F
:101B2A0006004001E4901B099312181D743A12181A
:091B3A001DD203755A0402198141
:0A1B43003098FDAF99C2987E002291
:1014DD00020922E493A3F8E493A34003F68001F2FA
:1014ED0008DFF48029E493A3F85407240CC8C33310
:1014FD00C4540F4420C8834004F456800146F6DFDF
:10150D00E4800B01020408102040809011CEE47E8F
:10151D00019360BCA3FF543F30E509541FFEE493D3
:10152D00A360010ECF54C025E060A840B8E493A39A
:10153D00FAE493A3F8E493A3C8C582C8CAC583CAC5
:10154D00F0A3C8C582C8CAC583CADFE9DEE780BE7D
:0111D7000017
:10178C00BB020689828A83E0224003BB0402E72263
:0B179C00400789828A83E49322E32245
:1017A700BB020689828A83F0224003BB0402F72228
:0417B7005001F322C8
:1017BB00FAE6FB0808E6F925F0F618E6CA3AF6222F
:1017CB00D083D082F8E4937012740193700DA3A3AD
:1017DB0093F8740193F5828883E4737402936860C1
:0617EB00EFA3A3A380DFC1
:101B4D00EFB40A07740D121B58740A309811A89936
:101B5D00B8130CC2983098FDA899C298B811F630F8
:071B6D0099FDC299F59922D0
:00000001FF
